:020000040000FA
:0E0000000219FDD2D3A68A08C2D332021223FF
:03001300020532B1
:0F001B00302F0AD2D3B284868B08C2D33281BB76
:10002B0075C800203E0653E6DF020417752741858D
:09003B0055CC8556CD43E6203278
:03005B000205405B
:10006300302456C521C59B30E61820181202041C03
:1000730053917FC050C05122759B80D2A08117C578
:100083002132C52120180132759100856C94856D4C
:10009300957550E8202410C56EF552047553E86039
:1000A3000375500014C56E75910443E680C218327F
:1000B300203E04D0E0012B8045759B80C0E0E59B8A
:1000C300652720E63120182B103821C2CA10CFE053
:1000D300E5CCF4F5CCE5CDF4F5CD303E0FC0D0C37F
:1000E300E5CC9555E5CD95564012D0D0B23ED2CA57
:1000F300D0E032D0E032D0E020188D32D0D0855518
:10010300CC8556CD80E6D0E075C80053E6DF811775
:100113000406080C10182030406080A0C0000000C6
:1001230000000000000000000000000000000000CC
:1001330000000000000000000000000000000000BC
:1001430000000000000000000000000000000000AC
:10015300000000000000000000000000000000009C
:10016300000000000000000000000000000000008C
:10017300000000000000000000000000000000007C
:10018300000000000000000000000000000000006C
:10019300000000000000000000000000000000005C
:1001A300000000000000000000000000000000004C
:1001B300000000000000000000000000000000003C
:1001C300000000000000000000000000000000002C
:1001D300000000000000000000000000000000001C
:1001E300000000000000000000000000000000000C
:1001F30000000000000000000000000000C55204E1
:1002030004700714C5528553503214C55232C2AF1D
:10021300C294D29575D536D2AF759F32754F24618E
:1002230059C2AF75D52DD2AF759F03754F33615941
:10023300C2AFC295D29375D52DD2AF759F31754F8D
:10024300466159C2AF75D51BD2AF759F23754F5504
:100253006159C2AFC293D29475D51BD2AF759F308B
:10026300754F686159C2AF75D536D2AF759F137597
:100273004F11D21A6159C2AFC295D29475D536D2F5
:10028300AF759F31754F8C6159C2AF75D51BD2AF16
:10029300759F03754F9B6159C2AFC294D29375D5B5
:1002A3001BD2AF759F32754FAE6159C2AF75D52D55
:1002B300D2AF759F13754FBD6159C2AFC293D2952B
:1002C30075D52DD2AF759F30754FD06159C2AF75BB
:1002D300D536D2AF759F23754F79D21A6159C21C97
:1002E300302406804BD21981177591008569948556
:1002F3006A957550E8202410C56BF552047553E8D0
:10030300600375500014C56B75910443E680C219F0
:10031300C21820200885D515853FD5D218752741E9
:10032300759BB075C8008555CC8556CD43E6203204
:10033300C2AF759100856994856A95759104D2AFB2
:100343007550E843E680C219D2187521807527419C
:1003530043E620020063302417C2AF759100856322
:1003630094856495759104D2AF7550E143E680326C
:100373007591008563948564957550E1202410C5BB
:1003830065F552047553E1600375500014C5657536
:10039300910443E680D21C3253E6DF75C8007591A1
:1003A30000856694856795854F50202410C568F5B0
:1003B3005204854F53600375500014C5687591044A
:1003C30043E680C0E0C0D0E55C64036038D21BE83C
:1003D300C557F8C3E5F9A660F56096F608E5FAA6F1
:1003E30061F56120DF0D96F608E54DA662F562968C
:1003F300F6807520E7F096F608E54D0480ED20E7DA
:10040300110562806D85F960E5FAF561854D62201D
:10041300DFEC805E20240A619B8515D5C521759B81
:1004230080C2AF759100856694856795759104D2F6
:10043300AF854F5043E68053E6DF75C800C0E0C088
:10044300D0E55C640360BED21BE8C557F8C3E5F989
:10045300A660F56096F608854D62E5FA20DF20A6D2
:1004630061F56196F6087600E8040444F0C557F890
:10047300055CE5245403600E2021020532801D2013
:10048300E7DD056280D9A218922730190F20230CCB
:10049300201809B177D226D0D0D0E032C3E55B95DE
:1004A30035400BD2A0C290C291C29275D53FD0D035
:1004B300D0E053E6DFC21932C2A8C0D0C0E0C28E7A
:1004C300D22D758A00E508B4B72E30332DD22FD242
:1004D3008443A4107508B9758921538EF0758B97E1
:1004E30085748C85738AC28DC28FD2BBD28CD28E17
:1004F30043A80AD0E0D0D032D22E85718B7508A7DD
:10050300D2A8D2AAD0E0D0D032E54E2418F54EE5D9
:100513002260021522C3E5396005753A00A12DE575
:100523003A2401F53A5003753AFFD0D0D0E032C2F5
:10053300AA85718BD28E85F94A85FA4B32C0E0E5E4
:10054300F730E61953F7DFE5F9E5FA30E10F853BBC
:10055300FB853CFC853DE9853EEA53F7BF10DF038D
:10056300D0E032C2DF054DC0D0E54E954D609AD044
:10057300D0D0E032C2AF75910075C800759B00D230
:10058300AFC2AFC290C291C292C293C294C29575D8
:10059300D53FD2AF227901801879038014790A807C
:1005A30010790F800C791E80087964800479C880E3
:1005B3000075A91375A71075C10075A70078147489
:1005C300F0000000D5E0FAD8F6D9F275A71075C18E
:1005D3003075A70075A9032279018014790380106F
:1005E300790A800C791E80087964800479C88000B8
:1005F30075910075949875954075910453E67FE95C
:10060300C0E0F1EFD0E0F9E59130E7F3D9E22278E9
:10061300FF20202879A1E76023E559601F74C48572
:1006230059F0848536F030210375F005A4F8C5F040
:10063300600278FFC3E895425002A842884122C372
:10064300E55D9400E55E9410E541500314800104D8
:100653006002F541220543C3E5439408404F30ED62
:10066300F475430079A0E76043E5BE7006E5446096
:1006730019800DC3E5BD9544600EE5445005600A3D
:100683001480070460FA8002E544F544C3954840AA
:100693001B7540C0C394044013754080C394044049
:1006A3000B754040C39404400375400022E5402489
:1006B30010500274FFF54022743279A687F0A4C566
:1006C300F0A2F733F54222755D00755EF0227A1CC5
:1006D3007B3C80127A147B4B800C7A107B5A800609
:1006E3007A0A7B788000EFD5E0012275A91375A7FC
:1006F3001075C10075A7007902E4C294D5E0FDD25C
:1007030091D5E0FDC291D5E0FDD294D5E0FDE9207D
:10071300E002D29030E002D292EFD5E0FDE920E092
:1007230002C29030E002C2927496D5E0FDD9CAEAC3
:10073300F8D5E0FDD8FBDBAEC29475A71075C130C8
:1007430075A70075A9032278867606087601789244
:100753007603087628087650087604087602087629
:1007630007087601087600087600227888E6C394A5
:1007730003D2325002C232C230E630E102D230A29A
:100783003092317886E6149001139378A6F6788632
:10079300E6F536C394025003753602789CE6753548
:1007A300FFB402037535A0B4030375358278A0E660
:1007B300F8600674282409D8FCF5482278A5E6F9E0
:1007C3005403C2857002D285E9540CC2867002D2EA
:1007D30086E95430C2877002D287E954C0C2B3702D
:1007E30002D2B322120C182212125622102DF5A295
:1007F3002BB033B02F40F122754600754700120528
:100803007775801F75F1F075A4E075801F75D4FFAF
:100813007590C075F23F75A53F7590C075D53F754E
:10082300A00075A60175A72075CC0175A700E5B5D5
:1008330025E0600975A71075CF0075A70075E34023
:1008430075E20212057712074A1213CC754C017533
:1008530057F07558F075510275A71075C13075A71B
:100863000075A903C2AF1205B0789886071206D1A6
:100873001205A41205A41205A41206D71205A41288
:1008830005A41205A41206DD1205A41205A412057F
:10089300A41206E31206E31205AC1207BF22C2AF8D
:1008A30053A4EFD28475A91375A71075C10075A75A
:1008B30000754600754700AAE475E4C478FA79FA2E
:1008C300308409D9FBD8F7021C008AE422C2A0C2F3
:1008D300AF12076E12057775A71075C13075A700A3
:1008E30075A903C22575D84075D90975F781759E19
:1008F3000375960275DA4275DB4275A82175E61019
:1009030043B801759B80759D3075D10C75BCB97565
:10091300BB1075E88075B20175340012059822305A
:10092300580675E44CD22B2275E4C4C22B22C2AF05
:1009330078988607A22B40071206E31206E32212D9
:1009430006DD1206DD22C2A0D2AF1205EF1205EBBF
:10095300C3E5399401400280EDC2AFA22B7898869B
:1009630007402CC0071206D1D2AF1205EBC2AFD09D
:10097300071206D1C007D2AF1205EBC2AFD00712E0
:1009830006D1C007D2AF1205EBC2AFD00780091260
:1009930006E31206E31206E3C289D2AF1205EF2281
:1009A300C2A0E4F55DF55EF55FF530F53175200025
:1009B30005203001457520000530E530F4703B0516
:1009C30031789AE67819146012783214600D787DC4
:1009D30014600878FA146003753100C3E531984058
:1009E3001912057712059815317530007899860725
:1009F300C2AF1206E3D2AF1205EB1205E3E5227094
:100A030002C3221205DB3028A7C3E5399401500A3B
:100A1300C3E56F9401501E0209B31205EBE5227082
:100A230002C322756F00757000D3227546A5754702
:100A3300F112140622AF6F12149F7546007547001A
:100A4300C22880BFC2A0C2AF7557F07558F0755C5D
:100A530000D2AF120577E4F543F523F524F55B7572
:100A630043081205DB75E89030EDFDA8BDE5BE70C7
:100A730001F888441206587543081206BB854240A4
:100A8300854241303207C230302902D230D220753C
:100A93003200E4C2AF85F96085FA61854D62D2AF59
:100AA300F55DF55E755F087559501210751211ECFE
:100AB30020300812028C12027980061202241202DC
:100AC3001175E890102613101B12102D5CA22BB089
:100AD30033B02F404F101A5680EA61E6D1A58563E3
:100AE30011856412121075202430E55924EC402A34
:100AF300C3E5639511F511E5649512F512401BC228
:100B0300AF301C16759100E5942511F594E59535E4
:100B130012F595759104D2AF4007D2AF1211EC8054
:100B2300A3759184121256809B120C188096202470
:100B330003120612302403120642120658302027ED
:100B430085424079187A0CC3E53299400EC220D20F
:100B5300218A33854240854241800CC3E5399401A3
:100B63004003020AC461EE30211F20231CE5331425
:100B73007006C221D22241C4F533203207C3E539BE
:100B830094014003020AC4806275340020320F7856
:100B9300FA79A4E760027803C3E53A98504DE52259
:100BA3006049303215203005202907800D30290295
:100BB3008008202305D22385424078F03023058521
:100BC30042407819C3E559985003020AC430231BE5
:100BD300C223C230302902D230D22175331285426A
:100BE3004041C40534E539600261F17534001205F2
:100BF30077752400C2891205EB12057775230078F7
:100C0300A4E66006D293D294D295C3E5349404400B
:100C130002C322D322102E0CE4AE72FCFBFA790835
:100C230078A78002A1D8E6FDC39CC39E40F69EEB45
:100C330033FB08E6FCC39DC39E40E99EEB33FB08F0
:100C4300E6FDC39CC39E40DC9EEB33FB08E6FCC37E
:100C53009DC39E40CF9EEB33FB08E6FDC39CC39E22
:100C630040C29EEB33FB08E6FCC39DC39E40B59E8A
:100C7300EB33FB08E6FDC39CC39E40A89EEB33FB0E
:100C830008E6FCC39DC39E409B9EEB33FB0880029A
:100C9300A1D8E6FDC39CC39E40F69EEA33FA08E65C
:100CA300FCC39DC39E40E99EEA33FA08E6FDC39C5C
:100CB300C39E40DC9EEA33FA08E6FCC39DC39E4014
:100CC300CF9EEA33FA08E6FDC39CC39E40C29EEA68
:100CD30033FA08E6FCC39DC39E40B59EEA33FA0887
:100CE300E6FDC39CC39E40A89EEA33FA08E6FCC314
:100CF3009DC39E409B9EEA33FA08EBC46B6A54F093
:100D0300F9EAC4302B01F454F0C3996002A1D8EB83
:100D1300F4C454F0F9EAF4C4540F49FAEBF4C4549C
:100D23000FFBC3EAF99460FAEB9400FB5020C3E98C
:100D33007B007A0079006016C3135006F9C3956FE0
:100D4300600AE9F56F757000790080020570303232
:100D530027C3EA94D0F8EB9407F9400BE8FAE9FBD0
:100D6300202909D2298005302902C229203102B263
:100D730029C3EA33FAEB33FBEB2B3B3BF9C3EB130E
:100D8300FBEA13FAEA29FAEB3400FB30E3047AFFB7
:100D93007BFFE5245403601B202218E54233F9EB63
:100DA3007007C3E99A4002E9FAE534C4332AFAEB3F
:100DB3003400FBC3EA33C4540FF8EB33C454F04894
:100DC300F87005EA60027801E579600215798024FC
:100DD30075220A80140579E57970021579C3E579DE
:100DE3009432500280EA753900202F07D2AAD2A884
:100DF3007508A722E830E702D2A08839D228E86034
:100E030003753A00C3E540FC95414002AC41C3EC95
:100E130095395008EC75F008A4FAABF0EBF4131312
:100E230092D5A2E75401F9EAF4FC13A2D513F8E52D
:100E33004C23F54CEC5403243783554C600BE824C6
:100E430001E9340020E10208F9C3E8940FFAE994B8
:100E530000FB50047A007B00883B893C8A3D8B3E33
:100E630075220A53F7DF43F740202F0343E610A10F
:100E7300EC00115577C3EC13FCEB13FBEA13FA8672
:100E83000508860608860708084300F08858C3EF5C
:100E9300941840027F18C3ED33FDEE33FEEF33FFAA
:100EA300E190A858302479AA5DAB5EC3EAC4540F1D
:100EB300FCEBC4FD54F04CCA9AFAED540FCB9BFBE8
:100EC300E60303543FFC08E60303FD54C04C2AFA2F
:100ED300ED543F3BFB0808084300F0D55CCDC21B33
:100EE30088587C008C5F8B5E8A5DECC40354F8F9F0
:100EF300EBC403540749F55978003027027801E51C
:100F03005B75F007A4F9E5F028F5F0E9A2F013A268
:100F1300F113A2F213F8C3947850027878885B2215
:100F2300AA5DAB5EAC5F302003020E78E559C39433
:100F330003400A94035003020FF0020FB7ECC4F905
:100F4300540FFFE954F0FEEBC4F9540F4EFEE9547D
:100F5300F0FDEAC4540F4DFDC3EA9DFAEB9EFBEC92
:100F63009FFC860508860608860708084300F08864
:100F730058EF0303F9543FFFE954C0CE0303F95478
:100F83003F4EFEE954C0CD0303543F4DFDEA2DFA15
:100F9300EB3EFBEC3FFC8C5F8B5E8A5DD55C13C242
:100FA3001BECC3941840097C18E4F55DF55E8C5F77
:100FB300C1EDC1A5EC0303F9543FFFE954C0FEEBB7
:100FC3000303F9543F4EFEE954C0FDEA0303543FC3
:100FD3004DFDC3EA9DFAEB9EFBEC9FFC860508865C
:100FE3000608860708084300F0885880A0ECC4234D
:100FF300F9541FFFE954E0FEEBC423F9541F4EFEDE
:10100300E954E0FDEAC423541F4DFDC3EA9DFAEB06
:101013009EFBEC9FFC8605088606088607080843A6
:1010230000F08858C3EF13FFEE13FEED13FD020F1C
:1010330090C3E55D2323F954FCFAE95403FBE55E11
:101043002323F954FC4BFBE95403FCE55F232354AE
:10105300FC4CFCC3E49AFAE49BFBE49CFC240C40A8
:1010630005E47CF4FAFBC2AF8A6C8B6D8C6ED2AF55
:101073008021E559600E147007C3E55E942D40048A
:10108300C22480ADD224C2AF756C98756D40756E65
:10109300FFD2AF3020057F030210A27892E6FFE56E
:1010A3005FC4FC540FFAEC54F0F9E55EC4FC540F32
:1010B30049F9EC54F0F8E55DC4540F48F8C3E894DB
:1010C30030FBE99400FCEA9400FD400CC3EB94016F
:1010D300EC9400ED940050057B01E4FCFD202047D7
:1010E300C3E49BF8E49CF9E49DFAE8FBE9FCEAFD20
:1010F300D3ED13FDEC13FCEB13FBC2AF8869896AD4
:101103008A6BD2AFC3EF94037065C2AF88668967F9
:101113008A68D2AF28F8EC39F9ED3AFAC2AF88639E
:1011230089648A65D2AF22E4C2AFF569F56A756B4B
:10113300FCD2AFC2AFF56CF56D756EFCD2AFC3E5F3
:10114300329401500FC2AF7563007564F87565FF83
:10115300D2AF800DC2AF7563007564F97565FFD2B8
:10116300AFC2AF7566007567FE7568FFD2AF222008
:10117300E111EB28F8EC39F9ED3AFAC3EF940340A7
:1011830016803DE828F8E939F9EA3AFA74FFFBFCDE
:10119300FDC3EF94035029C2AF886689678A68D27A
:1011A300AFD3E56B13FAE56A13F9E569132BFBE992
:1011B3003CF9EA3DFAC2AF886389648A65D2AF22FB
:1011C300C2AF8B668C678D68D2AFD3E56B13FDE539
:1011D3006A13FCE5691328F8EC39F9ED3AFAC2AF62
:1011E300886389648A65D2AF2220200430240C22CC
:1011F300C2AF7555217556FDD2AF227A807BFEE5CD
:1012030059C403F9530107F85300F8E9940140075F
:10121300E4C398FAE499FBC2AF8A558B56D2AF2246
:10122300C23353A4EFD2845388A5758C0075892AE1
:1012330085788E7508A785718BC2A9C2BBD2AAD245
:10124300A8D28CC22F32FBEA13FA0C803174FFFB55
:10125300FA8029E55FAB5EAA5DC403F85407FCE896
:1012630054F8CBC403F854074BFBE854F8CAC4033F
:1012730054074AFAEA24FFEB34FF50D1E4FCC3EBF2
:101283001370C3EC234B540FC4FBEAC4FA540F4B43
:10129300FBEA54F0FA6BC46B540F4A640FFA78B943
:1012A30074DAC0E07412C0E079757D13EA540F2438
:1012B3002A83C0E0C005EAC4540F241F83C0E0C0E2
:1012C30005EB540F241583C0E0C005EBC4540F2471
:1012D3000A83C0E0C005227600D23322000C1B240F
:1012E300303F4B5766727C8693A2AFBC0000000070
:1012F30000000000000000000000000000E7F60806
:10130300A67508A67708797522E7F608A67508A6D4
:101313007608A67508797522E7F608A67708797620
:1013230022E7F608A67708A67508797522E7F60876
:10133300A67508A67508A67608797522E7F608A6A5
:101343007608A67608797522E7F608A67608A675C4
:1013530008797622E7F608A67608A67508A6750822
:10136300797522E7F608A67508A676087976220924
:10137300E7F608A6770879752209E7F608A676083E
:1013830079762209E7F608A67608A6750879752204
:10139300E7F608A67508A67508A6750879762209E2
:1013A300E7F608A67508A6760879752209E7F60810
:1013B300A67508A6750879762209E7F608A67508C2
:1013C300A67508A67508797522901A0D78209132B2
:1013D300E520B4550AA39132E520B4AA0261F5755C
:1013E30046A57547F112074A9106754600754700F1
:1013F3008105901A0378807B269132A308DBFA904B
:101403001A2922C2AF91759152901A007403913731
:10141300A374009137A374219137901A0378807BCA
:10142300269136A308DBFA91889166901A2922E463
:1014330093F622E6438F01538FFDFFC3E583941C8C
:10144300400122EF8546B78547B7F0538FFE22430D
:101453008F02438F018546B78547B7901A0DF05326
:101463008FFC22901A0D74559137901A0E74AA911D
:1014730037227A3079807820901A409132E520F330
:1014830009A3DAF7227A307980901A40E391370979
:10149300A3DAF9227C051205B0DCFB22EFC3940723
:1014A300400FEFD3940E5009E570C394065002C366
:1014B30022EF14B40E0040030215599014CC75F0BA
:1014C30003A4C58325F0C583730214F60214F60240
:1014D30014F60214F60214F6021559021503021546
:1014E3001002151D0215280215590215560215334F
:1014F30002153DEF24FEFF7899E6FD12164F805644
:101503007F033032027F017888A60780407F043052
:1015130032027F027888A607802D30323978881608
:1015230016C232803120322E78880606D2328026C7
:101533007888E630E002800F8013901A0BE49364FE
:10154300017888F630E006D230D2318009C230C249
:10155300318003120A2EE4F56FF570D322E4F58887
:10156300780876A7C228F56FF570C2A975892AF5A0
:101573008DF58CC2AFD2AAD2AB757856758E5675DF
:101583008851C2AF7571E2757214C2AFD258120995
:10159300227573C17574FE7575FC7576F77577F1F1
:1015A30075790AD2AF1205EBE579C3940A5001228B
:1015B300C2AFC25812092275790AD2AF1205EBE500
:1015C30079C3940A5001227571C3757228C2AFD2D0
:1015D300581209227573FC7574FD7575F67576EBF3
:1015E3007577E075790AD2AF1205EBE579C3940AF2
:1015F300500122C2AFC25812092275790AD2AF1222
:1016030005EBE579C3940A500122C3227F08758153
:10161300CD43FF807597DE7597AD75EF06E4F5A9A9
:10162300F5A9AE070FA806E4F6EF70F61207FB1252
:1016330008A11208D012156050F512093112094998
:101643001209A350EA120A4740F680E38F088D0976
:10165300C2AF120577E50814601414601814601CF7
:101663001460192404701AAF091206D18013AF094C
:101673001206D7800CAF091206DD8005AF091206EA
:06168300E3D2AF0205EB0B
:1019FD0002160F030021FFFFFFFFFFFF06FF01FF90
:101A0D0055AA01FFFFFFFFFF03FFFFFF25D0285061
:0D1A1D0004FF02FF7AFF0701FFFF0000FF3A
:101A4000234A5F485F31352320202020202020209A
:101A500023424C48454C492445464D3842323123B7
:101A60002020202020202020202020202020202076
:101C0000C2AFC2D37597DE7597AD7581C075A90057
:101C100075A90043FF80752438752503B1DE752949
:101C2000A5752AF143F11053A4EFD28475D4FF7542
:101C3000E3407DFA780379E67C1075220075230075
:101C4000901DEB7B06752498752501308402814B2D
:101C5000208408D8FBD9F9DCF781BD308408D8FB93
:101C6000D9F9DCF781BDB19EE493A3C39A6004DD8A
:101C7000C381BDDBDBB190600281347B08E493FA61
:101C8000A3B171DBF87A30B171752200752300B110
:101C900090EAFCEBFDC3ED94FE400EB1908A278BD9
:101CA00028ED30E0048A828B83B1907AC270D8C369
:101CB000ED94FE601950CEBD0029EC600F75200038
:101CC0007521FF752900752A000200008100A827F0
:101CD000A9280809D804D90281E0B194EAF281D494
:101CE0000D81A9C3ED94035051EDA2E092007AC595
:101CF000C3E5829400E583941C508C200010438F30
:101D000002438F018529B7852AB7F0300027A8271D
:101D1000A9280809438F01538FFDD804D902A135A2
:101D2000C3E583941C4003A3A11AE28529B7852A41
:101D3000B7F0A3A11A538FFC81857AC1BD030CE4CF
:101D400093A3FAB155DCF8B14D81858187AA22AB06
:101D500023B171EBFAEA6222752608C3E52313F575
:101D600023E52213F52250066323A0632201D52622
:101D7000EAB1DEB1DE75260AEAF4200102D284302F
:101D80000102C284B1DEC3134002C201D526EB2298
:101D9000B194EAFB208402A194308402A1997526B3
:101DA00008AE24AF25C3EF13FFEE13FEB1E2B1DEA0
:101DB000C3EA133084024480FA30E703632201C38C
:101DC000E52313F523E52213F52250066323A063D0
:101DD0002201D526D9E52265236523F52222AE24EA
:101DE000AF250E0FDEFEDFFCD20122424C48656CAF
:091DF0006934373164E8B20601E0
:00000001FF
